:400000000010002011000000B5040000B504000010B500F06FFAC04670B5194C23688022D20213432360182000F020FC2268154B13402360144A154B1A602022144B1A602E
:400040001032144B1A60203A134B1A6082221206124B1A6000252560114A124B1A60124A124B1A60124A134B1A601349092000F0A3FB092000F08AFB104B1D6070BDC046A1
:4000800000010B40FFFFFBFF0600008004010B40080202401C0202403002024008010B40010000800000024002000080400002400F000080800002407D0A00000C020B40BA
:4000C00010B572B60122344B1A7000240FE033486200131959000B00411889881A5AC31858880004104300F043F90134E4B2012CEDD92A490C312A48403000F01FF9EE22E3
:400100001202284B1A60EE22274B1A6099231B04264A1360A021C902254A1160254A1360F0218903244A1160244A1360244A13600122244B1A600221234B1960234803787C
:400140003B32934314221343DBB20370204A107816230343DBB2137003231E4A13601E4A136006221D4802601D480260F6321D4802601D4802601D4A1160DB2109011C4AA3
:4001800011601C4A136024221B4B1A60FFF744FF00F004F910BDC0461C700F40EC1C00006C1D00000C0001401000014000500F4008500F4010500F4018500F4020500F4061
:4001C00030500F402000004000800F4001700F4000700F400000044018000440000104401801044000020440180204400003044008030440000404400804044010B5064C57
:400200002378002B07D1054B002B02D0044800E000BF0123237010BD58010020000000008C1C0000084B10B5002B03D00749084800E000BF07480368002B00D110BD064B1A
:40024000002BFBD09847F9E7000000005C0100208C1C0000C00000200000000010B500F069FA00F01DFA00F02BFA10BD70B5040000F080FA012000F0D7FA9620400000F068
:40028000EBFA022000F026FA002000F037FA084D64006053642100F0ABFF02B26253054C0549200001F0C4F8200000F045FA70BDD4010020AC010020901C000010B5044A89
:4002C00000210A2000F0D8FC00F040FC10BDC046E8010020002306E05900044A895E044AD1540133DBB2092BF6D97047D4010020E801002010B562B6FFF7B0FFFFF7DEFF0F
:4003000000F028FA002404E02000FFF7AFFF0134E4B2092CF8D9074B1B789A0705D502229343044A1370FFF7D5FF034800F004FAE8E7C04674010020981C0000F0B50025F8
:40034000002711E0BB00C658F3B2FF22964308E06A008A181478A419527822700135013BDBB2002BF4D10137072FEBD9F0BDC04610B50A00002101F053F810BD064B1B68B3
:40038000002803D080221206134301E05B005B08014A13607047C04680031A4010B58022D202034B1A600120FFF7E8FF10BDC04600031A40092833D880001A4B1B589F4691
:4003C0004022194B1A602BE08022174B1A6027E02022154B1A6023E01022134B1A601FE0124A116806230B43136019E0104A116860230B43136013E00C4A116860230B43A3
:4004000013600DE00A4A1368C021C9000B43136006E00422044B1A6002E00822024B1A607047C0469C1C000000031A400000014004000140092832D88000194B1B589F46AB
:400440004022184B1A602AE08022164B1A6026E02022144B1A6022E01022124B1A601EE0114A136806218B43136018E00F4A136860218B43136012E00B4A136860218B43AF
:4004800013600CE0094A1168094B0B40136006E00422044B1A6002E00822024B1A607047C41C000004031A400000014004000140FFF9FFFF10B500F087FF03680C2B00D135
:4004C000FEE7FEE710B50300084A1068C318084A9A1A802A02DC054A136005E000F074FF0C2303600120404210BDC046C40000201002002070B50F4E0F4D13E029686B68DA
:40050000AC68002202E001C901C30432A242FAD1E868002202E0002102C304328242FAD11035013E002EE9D100F054FFFFF7E2FEFEE7C04601000000541E000010B5002366
:400540000AE0032B03D89A000949505800E009489900094A885001332F2BF2D9FFF7B0FD8022D205116801230B43136010BDC04600000000B50400000000002010B5032197
:400580000E2000F02BF924490E2000F015F90122224B1A60224B1B68002B01DA214900E02149224A13680B431360214A214B1A60214A224B1A600023214A1360214A22498A
:4005C0000A6022490A6022490A688020400202430A60204A1360204A136001331F4A136002211F4A11601F4908681F4A024013430B6000230DE09A001C4951188020C0006B
:400600000860580000241A4944521A481A4950500133002BEFD010BD2907000020001A4080031A40400210534002005300001A40C500008004001A400000FF0718001A4057
:400640001C001A400200020010001A4014001A4000031A4028021A4038021A4018021A40000F1A4030001A40FFFFFFDF80001A40F8010020204E0000F401002010B5074BE3
:400680001B68002B08DB054A1368802109060B4313600A2000F0E0F810BDC04600001A4010B5064B1B78002B04D1FFF767FF0122024B1A70FFF7E2FF10BDC046760100200F
:4006C000034A1368802149020B4313607047C04604001A40020083070CD0074B1B680120184001D19307F8D4002804D00122024B1A6000E00020704710021A4010B5041E8C
:4007000002D0002000F056F8002C07D1A400054B9C46644420680004000C00E0002000B210BDC04680011A40014B1A681A60704710021A407047C04670B505000078012420
:4007400004E000F04DFC285D0134E4B20028F8D170BDC04610B5002404E02000FFF76AFE0134E4B2092CF8D9FF22014B1A7010BDD400002010B50400FFF7ECFF2000FFF754
:4007800019FE014B1C7010BDD40000201F2318401E3B8340014A13607047C04600E100E01F2318401E3B8340014A13607047C04680E100E001BE704770B504000D001F2832
:4007C00002D90020FFF7F6FF1034A40080239B059C4664442068256070BDC04670B504000E00032902D90020FFF7E4FF1F2C02D90020FFF7DFFF03252540ED00063500F028
:4008000065FCA408A400074B9C46644421680323AB4099430B003100A9401943216000F059FC70BD00E400E010B5040006E0084B586800F041FC074B9C46644480231B02F2
:400840009C42F4D8024B9868604300F035FC10BDD80000200080FFFF10B5034B1B7B584300F02AFC10BDC046D8000020F0B557464E46C0B483B0040000F028FC0190E71E2A
:400880002D2F74D83F4B1B78DBB29C4208D83E4B1B78DBB29A463D4B1B78DBB2994631E03B4B1B78DBB29C4208D83A4B1B78DBB29A46394B1B78DBB2994623E0374B1B7883
:4008C000DBB29C4208D8364B1B78DBB29A46354B1B78DBB2994615E0334B1B78DBB29C4208D8324B1B78DBB29A46314B1B78DBB2994607E02F4B1B78DBB29A462E4B1B78F7
:40090000DBB299462D4BDE5D2F2E09D92A2C07D919222B4B1A60052000F0CEFB192503E0274B1D683F231D40B54206D9234BDA5D234B1A60052000F0BFFB1F4B9C4664441D
:400940002378DBB21F4A13601F4B52461A601F4B4A461A600520FFF77FFFB5420AD2174BDA5D174B1A60052000F0A6FB02E00020FFF720FF019800F0ADFB03B00CBC914652
:400980009A46F0BDC0F1FF0FC1F1FF0FC2F1FF0FC3F1FF0FC4F1FF0FC5F1FF0FC6F1FF0FC7F1FF0FC8F1FF0FC9F1FF0FCAF1FF0FCBF1FF0FCCF1FF0FCDF1FF0FCC1D0000F4
:4009C0002CFF0B4028FF0B401CFF0B4020FF0B40034B1868C0231B02184000D00120704700010B4010B500F071FB044A1368C02109020B43136000F06DFB10BD00010B401D
:400A000010B500F063FB08490A68084B1A408024E40122430A600A6813408022120213430B6000F057FB10BD00010B40FF3FFFFF70B5050000F04AFB0400FFF7C9FF0028BF
:400A400003D0FFF7DDFF012100E0002108482840084A1568084B2B40184310601368012901D1FFF7BFFF200000F034FB70BDC0460404040010020B40FBFBFBFF10B5244B74
:400A80001B685B0715D5234B1B685B070ED5224BD969042001401F4C22688A432260DA698243DA611B69002B00D098470420FFF7BFFF174B1B685B0518D5164B1B685B05EA
:400AC00010D5154BD9698022D2001140114802688A430260D969114A0A40DA615B69002B00D098478020C000FFF7A2FF084B1B685B030CD5074B1B685B0304D5064B9B698B
:400B0000002B00D098478020C002FFF791FF10BD10020B40EC00002078010020FFFBFFFF10B50A20FFF732FE10BDC04610B500F03BF810BD10B5044A1368802109060B4303
:400B40001360FFF7EDFF10BD0000064010B5064B1B78002B04D1FFF7E9FF0122024B1A70FFF7E8FF10BDC046980100200A4B1B68DB050DD5094B1B685B0409D4064B1968A4
:400B8000074A0A401A601A68802149000A431A600222044B1A6070470000064060000640FFFEFFFF6C00064010B500241C4B1C601C4A1D4B1A601D4A11680C230B431360CC
:400BC0001B4B1C4A13601C4A14601C491C4A11601C4A13601C4B1C600A20FFF7E1FD03210A20FFF7FBFD19490A20FFF7E5FD184B1C60184B1C605222FF32174B1A60174BA5
:400C00001C60174B1C60174B1C60174B1C70174B1C70174B1C80174B00221A7010BDC046000006400008004060000640700006400701008000030640040306402000FE009B
:400C4000100306400002064004020640A90C0000C80E0640880E0640480F0640080F0640C80F0640880F0640FC010020FD010020040200200002002070B506000D00141EF9
:400C80000BD00A20FFF78CFD044B1C60044B1E80044B1D800A20FFF779FD70BD08020020FE0100200202002070B5AC4B1B68002B00D09847AA4B1C88AA4B1D68AA4B1E68D5
:400CC0000223FF331D4242D0A84A13685B005B081360A74B1B789B0620D5A54A137820218B431370117810230B43DBB21370A14B1B68DB060CD4A04B1A78994B1B889A423D
:400D00000CD09B4A117808230B43DBB2137005E0974A117802230B43DBB21370974A1168974B0B4013600023964A1360914A13609549964A116096498A4A1160954A13709B
:400D40008A4A1368802109060B43136003E1F30602D50022904B1A600A23334200D190E08E4B1B685B0756D58D4B1B68894A1278002A16D0012A47D18A4A1288002A0DD03C
:400D80000121894A1160894A12681219DBB213700134844A1388013B138038E0FFF7E6FE35E0834A128893422BD201217E4A1160804A1288934202D2D21A92B200E00022FE
:400DC00078490A80072A03D80121724A117014E0082A09D169490A68A020000202430A600021684A116008E064490A688020800102430A600821634A11605F4A13701C00FE
:400E000005E0FFF7B3FE02E00020FFF7D3FC04225E4B1A6035E0594B1B689B0431D5B3070DD5654B1B680F211940544A1068544B03401360012014E00821012011E0594B7E
:400E40001988083989B219800829F5D8002008E0564B1B681B19524A1268D2B21A70013401390029F4D1002808D1444A1368802109020B4313600022424B1A600C22434B81
:400E80001A60B30746D5EB0615D500233D4A1360384A1360384B1B789C4201D1022300E00A232B40324A11780B4320218B4313700022384B1A706B062AD52D4A11782023CC
:400EC0000B43DBB213702C4B1B781C003B4A1268D20612D5364A1288D31A324A1380384B1A68802149020A431A601968354A0A401A6010221F4B1A6002E00422214B1A601A
:400F00000123314A13602249164A1160264A1360144B1D60144B1B685B071CD5214B1B88002B0CD0214B1B681B191B78DBB2274A136001341B4A1388013B138002E0FF222B
:400F4000224B1A60224B1B680F221340082BE5D10132204B1A60024B1C8070BD9C01002004020020400F0640000E064000000640FD010020880F064000020020600006402A
:400F8000FF5FFFFFC80F0640ED0F0000C00F0640FF0F0000FC010020880E0640CC0F064040030640A00100206C00064008020020FE0100200202002008030640640006401B
:400FC00004020640FFFFFEFF800E06404002064008020640800F06400000000000000000FEB5494652465B460EB407462E4909688A462E4A12682E48022100F06FF8030002
:401000002A480068C0182A4900F068F806001F3EB346234A126801219140C9430C000125002600F053F8814651460B6823400B605846043000F040F83800F040284090402D
:401040000B68234003430B60584600F035F80136072EF1D900200130012090400B68234003430B605846063000F026F8484600F031F8C046C046C0460EBC894692469B4642
:40108000FEBDC046C046C046C046C046C046C046C046C046C046C046C046C046C046C046D0000020CC000020C8000020E800002000C20100000000000230800804D0C046F8
:4010C0000138FDD1C046C046C0467047EFF3108072B6704780F310887047C046002243088B4274D303098B425FD3030A8B4244D3030B8B4228D3030C8B420DD3FF220902CC
:4011000012BA030C8B4202D31212090265D0030B8B4219D300E0090AC30B8B4201D3CB03C01A5241830B8B4201D38B03C01A5241430B8B4201D34B03C01A5241030B8B42BB
:4011400001D30B03C01A5241C30A8B4201D3CB02C01A5241830A8B4201D38B02C01A5241430A8B4201D34B02C01A5241030A8B4201D30B02C01A5241CDD2C3098B4201D374
:40118000CB01C01A524183098B4201D38B01C01A524143098B4201D34B01C01A524103098B4201D30B01C01A5241C3088B4201D3CB00C01A524183088B4201D38B00C01ACF
:4011C000524143088B4201D34B00C01A5241411A00D20146524110467047FFE701B5002000F0F0F802BDC0460029F7D076E7704703460B437FD4002243088B4274D30309D0
:401200008B425FD3030A8B4244D3030B8B4228D3030C8B420DD3FF22090212BA030C8B4202D31212090265D0030B8B4219D300E0090AC30B8B4201D3CB03C01A5241830B2D
:401240008B4201D38B03C01A5241430B8B4201D34B03C01A5241030B8B4201D30B03C01A5241C30A8B4201D3CB02C01A5241830A8B4201D38B02C01A5241430A8B4201D340
:401280004B02C01A5241030A8B4201D30B02C01A5241CDD2C3098B4201D3CB01C01A524183098B4201D38B01C01A524143098B4201D34B01C01A524103098B4201D30B0182
:4012C000C01A5241C3088B4201D3CB00C01A524183088B4201D38B00C01A524143088B4201D34B00C01A5241411A00D201465241104670475DE0CA0F00D04942031000D3AA
:401300004042534000229C4603098B422DD3030A8B4212D3FC22890112BA030A8B420CD3890192118B4208D3890192118B4204D389013AD0921100E08909C3098B4201D313
:40134000CB01C01A524183098B4201D38B01C01A524143098B4201D34B01C01A524103098B4201D30B01C01A5241C3088B4201D3CB00C01A524183088B4201D38B00C01A0D
:401380005241D9D243088B4201D34B00C01A5241411A00D20146634652415B10104601D34042002B00D54942704763465B1000D3404201B5002000F005F802BD0029F8D066
:4013C00016E770477047C046014B18687047C046500100200E4B70B500251E000D4CE41AA410A54204D0AB00F35898470135F8E700F01EFD084B00251E00084CE41AA4106A
:40140000A54204D0AB00F35898470135F8E770BD3C1E00003C1E00003C1E0000441E000003008218934202D019700133FAE770470EB410B59DB002A9029008610B4882245E
:4014400088604861012040421FABC881084804CBA400006801938C8100F06EF80023029A13701DB010BC08BC03B01847FFFFFF7F50010020F0B58E6885B007000C000392ED
:4014800001939E4243D890238A89DB001A423ED003250969236801985B1A029363695D43EB0F5D19029B6D1001331B18AB4200D91D00530510D52900380000F041FB061E9C
:4014C00014D0029A216900F0D0FAA289194B134080221343A38112E02A00380000F090FB061E0CD12169380000F0DEFA0C23402201203B60A38940421343A38117E0029BC7
:401500002661F61826606561019EED1AA560019BB34200D21E0032000399206800F0AEFA0020A3689B1BA36023689E19266005B0F0BDC0467FFBFFFFF0B59FB00290059306
:401540008B890F0016001B0610D50B69002B0DD1402100F0F5FA38603861002804D10C23029A01381360D8E040237B61002306AD6B6120336B761033AB7634002378002B9F
:4015800003D1A31B049312D003E0252BF9D00134F4E7A31B320039000298FFF76BFF431C00D1B4E06A69049B944663446B612378002B00D1ABE00122002352426A6002A9FD
:4015C0005432521801342B60EB60AB601370AB65534E21780522300000F03CFA002807D00123801B83402A68013413432B60EFE72B68DA0604D55322202102A81218117045
:401600001A0704D553222B2102A81218117022782A2A03D0099B00200A210EE0059A111D12680591002A01DB099204E05242EA60022213432B6001340BE02278303A092A60
:4016400004D84B4301349B180120F6E7002800D0099323782E2B1ED163782A2B0AD1059B02341A1D1B680592002B01DA01235B42079310E000230A201A0001346B60217820
:401680003039092904D84243013452180123F6E7002B00D00792234E21780322300000F0D9F9002806D04023801B83402A68013413432B60217806221B48661C297600F03D
:4016C000C9F9002812D0194B002B06D10722059B073393430833059314E005AB00933A00134B2900029800E000BF07E005AB00933A000F4B2900029800F08AF80390039BB7
:40170000013304D06B69039A9B186B6135E7BB890B985B0601D5012040421FB0F0BDC046FC1D0000021E0000061E00000000000075140000F7B5170001938A680B6900901F
:401740000C00934200DA130022003B6043321278002A01D001333B6023689B0602D53B6802333B60062523681D401ED0230043331B785A1E9341226892061CD53020E118CA
:401780004331087021005A1C45310978A2184332023311700FE022000123193201990098089EB047431C0ED00135E3683A689B1A9D42F0DBDAE72200019943320098089D8D
:4017C000A847431C02D10120404220E006232068E1683A6803400025042B03D18D1AEB43DB171D40A3682269934201DD9B1AED180027BD420AD0220001231A320199009833
:40180000089EB047431CDED00137F2E70020FEBDF0B58BB006920A0043320793059004920A7E0C00109B6E2A00D1ABE011D8632A22D009D8002A00D1B5E0582A00D0C5E053
:4018400045310A70814A4FE0642A1DD0692A1BD0BCE0732A00D1AAE009D86F2A29D0702A00D0B3E0202209680A43226037E0752A1FD0782A33D0A9E00E001A684236111DF6
:40188000196013683370A4E021681A68080606D4490604D5111D19600023D55E02E0111D19601568002D3BDA2D23049A6D42137036E021681A68080606D4490604D51568DF
:4018C000111D1960ADB202E0111D196015685F4B227E039308276F2A1DD00A271BE022007821453211705A4A19680392081D226818600D68100602D4500600D5ADB2D307C2
:4019000002D520231A4322601027002D03D1202322689A4322602300002243331A7002E00A274A4B03936368A360002B09DB0422216891432160002D05D1049E002B11D035
:401940007BE0002D79D0049E28003900FFF74CFC039B013E5B5C280033703900FFF7BEFB051EF1D1082F09D12368DB0706D563682269934202DC3023013E3370049B9B1B3D
:4019800023612BE009681A68080607D4490605D5111D19601368A28A1A8004E0111D1960136862691A600023049E236116E01A68111D1960166800216268300000F04AF82D
:4019C000002801D0801B6060636803E0260042363270012323610023049A1370079B09AA00932100069B0598FFF7A4FE431C02D10120404227E02369320006990598079D60
:401A0000A847431CF4D0236800259B070FD4099BE068984217DA180015E022000123193206990598079EB047431CE1D00135E368099A9B1A9D42F0DBE9E72600039B423693
:401A40001B7833708EE70BB0F0BDC0460D1E00001E1E0000C9B28218904204D003788B4202D00130F8E700207047002310B59A4203D0CC5CC4540133F9E710BD10B58842E3
:401A800002D98B18984201D3002305E09B1A013A08D3995C8154FAE7934203D0CC5CC4540133F9E710BD000070B50500002944D00C1F2368002B00DAE418280000F0D8F8AD
:401AC0001E4A13681100002B02D16360146031E0A3420DD92268A018834203D118685B688218226063600C6024E0A24203D813005A68002AF9D11E689819A0420BD121686E
:401B0000711858181960824214D110685268411819605A600EE0A04202D90C232B6009E021686018824203D1106852684118216062605C60280000F09CF870BDA8010020B9
:401B4000032370B5CD1C9D43083506000C2D01D20C2501E0002D01DBA94202D90C23336048E0300000F084F8234B1C681A002100002913D00B685B1B0DD40B2B02D90B601C
:401B8000CC181EE08C4202D1636813601AE04B6863600C0016E00C004968E9E7174C2368002B03D1300000F051F820602900300000F04CF8431C18D00323C41C9C43A042F4
:401BC0000DD12560300000F054F8200007220B30231D9043C31A0ED05A42E2500BE0211A300000F033F8431CEBD10C233000336000F03FF8002070BDA8010020A401002076
:401C0000F8B506000C001500002904D11100FFF797FF040018E0002A03D1FFF745FF2C0012E000F027F885420ED929003000FFF787FF071E07D021002A00FFF716FF2100DE
:401C40003000FFF731FF3C002000F8BD002370B5064C050008002360FEF734FC431C03D12368002B00D02B6070BDC0460C020020704770470B1F1A68101F002A04DA891817
:401C800004390B68D018043870470000000000002533642C202000000D0A0000C0030000C8030000D0030000D8030000E0030000EC030000F8030000040400001204000033
:401CC0001A04000040040000480400005004000058040000600400006C0400007804000084040000900400009804000000300F40000400400F400004830DB601BE40D80447
:401D0000DF011F808308404549FF4AFF4BFF4F0150185A045F016040624064406540668068806A806C806E808E019201B001B201BE01C054C5ECC720C823C9FFCAFFCBFF6F
:401D4000CD83CE03CF01D018D280D401D804DA04DB04DF01E040E240E440E540E680E880EA80EC80EE8002020B401A401B084101468049054B404E025101520259055A40B2
:401D800072807340A708AF80C001C208D081D218D60B57206C048004D440DA80E6805701A301AF21D620EE100101100101000F4004300F4002310F4030320F4016330F4049
:401DC00006400F4005410F4002600F40030405060708090A0B0C0E0F101112131415161718191B1C1D1E1F2021222325262728292A2B2E2F3031323334354300232D302B2A
:401E00002000686C4C00656667454647003031323334353637383941424344454600303132333435363738396162636465660000F8B5C046F8BC08BC9E467047250200006D
:401E40003D050000F8B5C046F8BC08BC9E467047FD010000681E0000C000002098000000B8000000000000000000000010020020000304400300000001000000FF0000002A
:401E8000010000000000E02EC05D00001800000000366E01040404000000000000000000000000000000000000000000000000000000000000000000FA1D00000000000016
:401EC0000000000000000000000000000000000000000000000000000000000000000000000000000000000000000000000000000000000000000000F000002000000000D2
:401F000000000000000000000000000000000000000000000000000000000000000000000000000000000000000000000000000000000000000000000000000000000000A1
:401F40000000000000000000000000000000000000000000000000000000000000000000000000000000000000000000000000000000000000000000000000000000000061
:401F80000000000000000000000000000000000000000000000000000000000000000000000000000000000000000000000000000000000000000000000000000000000021
:401FC00000000000000000000000000000000000000000000000000000000000000000000000000000000000000000000000000000000000000000000000000000000000E1
:0200000490303A
:020000009EE57B
:0200000490402A
:200000000000000000000000000000000000000000000000000000000000000000000000E0
:0200000490501A
:0C000000000204A61193110104AFB078B7
:0200000490600A
:0100000001FE
:00000001FF